:1000000012C01895A9C118951895189518951895A6
:10001000189563C218951895189518951895189500
:100020001895189518958FE58DBFC8E3E0E24E2E20
:1000300084E08EBFD4E0F4E05F2EA89584B7082E4C
:10004000877F84BF88E1992781BD91BDEEEFF3E002
:10005000A0E6B0E088278D933197E9F7662472EB2C
:1000600071BF8FEF87BB8FEF81BB80E084BB8C9823
:100070008B9883E886B980EC87B982E083BF85B727
:10008000837F886085BF79B7716079BF7BB77068FF
:100090007BBF80E08093830080E08093840080E0D9
:1000A00090E0A5E8B0E08D939C9380E090E0A7E815
:1000B000B0E08D939C937894A5E8B0E08D919C91ED
:1000C000ADE6B0E08D939C939A9901C0FDCF83E09B
:1000D00090E087D3379AAFE7B0E08D919C91A1E88B
:1000E000B0E08D939C93ADE7B0E08D919C91AFE72C
:1000F000B0E08D939C93ABE7B0E08D919C91ADE720
:10010000B0E08D939C93A9E7B0E08D919C91ABE713
:10011000B0E08D939C93A7E7B0E08D919C91A9E707
:10012000B0E08D939C93A5E7B0E08D919C91A7E7FB
:10013000B0E08D939C93A3E7B0E08D919C91A5E7EF
:10014000B0E08D939C9307B1007F066007B958D348
:10015000A3E7B0E08D939C93A3E7B0E00D911C91D1
:10016000A5E7B0E04D915C91040F151FA1E7B0E049
:100170000D931C93A1E7B0E00D911C91A7E7B0E0AF
:100180004D915C91040F151FA1E7B0E00D931C93F6
:10019000A1E7B0E00D911C91A9E7B0E04D915C9111
:1001A000040F151FA1E7B0E00D931C93A1E7B0E089
:1001B0000D911C91ABE7B0E04D915C91040F151FC0
:1001C000A1E7B0E00D931C93A1E7B0E00D911C9165
:1001D000ADE7B0E04D915C91040F151FA1E7B0E0D1
:1001E0000D931C93A1E7B0E00D911C91AFE7B0E037
:1001F0004D915C91040F151FA1E7B0E00D931C9386
:10020000A1E7B0E00D911C91A1E8B0E04D915C91A7
:10021000040F151FA1E7B0E00D931C93A1E7B0E018
:100220000D911C9148E050E0B9D2A1E7B0E04D93A8
:100230005C93929AEF93E2E0EA95F1F7EF9192984E
:1002400084990CC0A1E7B0E08D919C91ABE6B0E041
:100250008D939C9384E690E0C4D278C0A3E8B0E08C
:100260008C918F5F8C9300918300023310F009F022
:1002700001C067C0A4E8B0E08C918F5F8C9381E0EF
:1002800080938300009184000C3310F009F001C0CA
:1002900058C0E2E1F0E0A0E1B0E0E7D20C5E1F4F11
:1002A000AFE6B0E00D931C93AFE6B0E04D915C91EA
:1002B000A1E7B0E00D911C910417150710F009F0AB
:1002C00001C012C0A5E8B0E03FD2E4E1F0E0A9E649
:1002D000B0E0CBD2A9E6B0E037D2E4E1F0E0A9E6A5
:1002E000B0E07BE7B1D22AC0E0E1F0E0A0E1B0E00D
:1002F000BCD204511040AFE6B0E00D931C93AFE6C2
:10030000B0E04D915C91A1E7B0E00D911C91041714
:10031000150710F009F001C011C0A7E8B0E014D231
:10032000E6E1F0E0A9E6B0E0A0D2A9E6B0E00CD2A8
:10033000E6E1F0E0A9E6B0E07BE786D281E08093D9
:100340008400E4E1F0E0ABE6B0E08FD29A9B01C01C
:10035000FDCFBACEF894FFCF0F921F922F923F920B
:100360004F925F927F92AF92BF920F931F932F9302
:100370003F934F935F936F937F938F939F93AF932D
:10038000BF93CF93DF93EF93FF938FB78F9379B79B
:10039000716079BF789483997FC080E080938900F1
:1003A000849931C0E0E1F0E0AFE6B0E05ED2AFE6C4
:1003B000B0E04D915C91ABE6B0E00D911C9104175B
:1003C000150708F006C0E0E1F0E0ABE6B0E07BE73F
:1003D0003BD2E2E1F0E0AFE6B0E047D2AFE6B0E01A
:1003E0004D915C91ABE6B0E00D911C91041715079F
:1003F00010F009F001C006C0E2E1F0E0ABE6B0E0C9
:100400007BE722D205C0E6E1F0E0ABE6B0E02DD21A
:10041000839942C084E690E0E4D1A9E8B0E08C91F1
:100420008F5F8C9300918900023310F009F001C0B6
:1004300032C079B77E7F79BF849911C0E0E1F0E0E6
:100440000CED10E0A0E1BB277BE7FED1E2E1F0E09C
:1004500008E210E0A0E1BB277BE7F6D11CC080E0FA
:1004600090E0A7E8B0E08D939C9380E090E0A5E851
:10047000B0E08D939C93E4E1F0E000E010E0A0E1B7
:10048000BB277BE7E1D1E6E1F0E000E010E0A0E18E
:10049000BB277BE7D9D1BCCF79B7716079BF70E456
:1004A0007ABF8F918FBFFF91EF91DF91CF91BF9175
:1004B000AF919F918F917F916F915F914F913F91FC
:1004C0002F911F910F91BF90AF907F905F904F90B1
:1004D0003F902F901F900F9018950F921F922F9280
:1004E0003F924F925F927F92AF92BF920F931F9372
:1004F0002F933F934F935F936F937F938F939F932C
:10050000AF93BF93CF93DF93EF93FF938FB78F9307
:10051000882783BF80E080936600ABE6B0E08D91D2
:100520009C91ADE6B0E08D939C93ADE6B0E00D916B
:100530001C91033650E0150710F009F001C010C0FF
:10054000A6E6B0E08C918F5F8C93ADE6B0E00D91A4
:100550001C9104561040ADE6B0E00D931C93E5CF1E
:1005600080E080936500ADE6B0E00D911C9109300C
:1005700050E0150710F009F001C010C0A5E6B0E08A
:100580008C918F5F8C93ADE6B0E00D911C910A5079
:100590001040ADE6B0E00D931C93E5CF80916D0067
:1005A00080936400979896989598A0E6B0E08C9117
:1005B0008F5F8C9300916000033010F009F001C050
:1005C00003C081E08093600080E08093620074D07B
:1005D000A1E6B0E08C9180FBA8E3B0E08C9187F9B4
:1005E0008C936AD0A1E6B0E08C9180FBA8E3B0E0E8
:1005F0008C9185F98C9360D0A1E6B0E08C9180FB62
:10060000A8E3B0E08C9183F98C9356D0A1E6B0E0DA
:100610008C9180FBA8E3B0E08C9181F98C934CD055
:10062000A1E6B0E08C9180FBA8E3B0E08C9180F96A
:100630008C9342D0A1E6B0E08C9180FBA8E3B0E0BF
:100640008C9186F98C9338D0A1E6B0E08C9180FB38
:10065000A8E3B0E08C9184F98C93C29A0091600079
:10066000013009F002C0979A09C0023009F002C0B7
:10067000969A04C0033009F001C0959A82E083BFC6
:100680008F918FBFFF91EF91DF91CF91BF91AF918C
:100690009F918F917F916F915F914F913F912F919A
:1006A0001F910F91BF90AF907F905F904F903F90C0
:1006B0002F901F900F901895A0E6B0E0AD90BB244E
:1006C000A3E6B0E0AA0DBB1D0C9147E0049FA1E694
:1006D000B0E00C920091620040916100040FA1E62D
:1006E000B0E00C93E2E0F7E0A1E6B0E08C9199274E
:1006F000A1E6B0E09ED0A2E6B0E08C918F5F8C9333
:100700000895000000000000010100000101010146
:1007100000000100000100000000000101000100D4
:1007200000010100000001000001000000010000C4
:1007300000000000000001010101000000000000B5
:100740000000000000010000ED91FC91EF5FFF4F01
:10075000FC93EE93089500FC10D0089503D01ED0B2
:1007600001F8F9CF0024E89457FF02C009D068943B
:1007700000F80BD010F80124089502D009D0089594
:10078000509540954F5F5F4F0895E89417FF089587
:10079000009510950F5F1F4F68940895352F242FF3
:1007A000E894452B11F468940895512F402F0027A9
:1007B000112780E1440F551F001F111F021B130B4F
:1007C000416018F4020F131F4E7F8A9599F7089520
:1007D0003197F1F70895689462F80895E89462F803
:1007E0000895EF93FF93EE27E82BE92B31F0EAEF22
:1007F000F0E03197F1F70197D1F7FF91EF9108956C
:10080000369A3699FECF369A3699FECF84B195B195
:100810000895C89531960020089591E005C092E0B2
:1008200003C094E001C098E0F4DF0D929A95E1F7DF
:100830000895E80FF91FF1CFE199FECFEEBBFFBBA2
:100840003196089591E001C092E07B3751F47FB773
:10085000F894F2DF8D918DBBE29AE19A9A95C9F7EF
:100860007FBF7727089591E001C092E0E5DFE09A2D
:0A0870008DB38D939A95D1F708958A
:00000001FF
